:020000040800F2
:10000000B8080020FD190008B1060008B306000872
:10001000B7060008BB060008BF0600080000000085
:10002000000000000000000000000000C3060008FF
:10003000C506000800000000C7060008C906000841
:10004000171A0008171A0008171A0008171A0008CC
:10005000171A0008171A0008171A0008171A0008BC
:10006000171A0008171A0008171A0008171A0008AC
:10007000171A0008171A0008171A0008171A00089C
:10008000171A0008171A0008171A0008171A00088C
:10009000171A0008171A0008171A0008171A00087C
:1000A000171A0008171A0008171A0008171A00086C
:1000B000171A0008310C0008171A0008171A000850
:1000C000171A0008171A0008171A0008171A00084C
:1000D000171A000871190008171A00088D0900087E
:1000E000171A0008171A0008171A0008DFF80CD0B2
:1000F00003F0F6F90048004703040008B8080020A0
:1001000070B505460C46164654B904EBC40205F119
:10011000300101EB82003246FDA103F021FA18E024
:10012000012C0AD104EBC40205F1300101EB82007D
:100130003246FBA103F014FA0BE0022C09D104EBC8
:10014000C40205F1300101EB82003246F7A103F051
:1001500007FA04EBC40105F1300000EB81000662F0
:1001600070BD10B50A220021F448FFF7C9FF0A222A
:100170000121F248FFF7C4FF0A220221EF48FFF7EE
:10018000BFFF0720ED49C8600020086148610022D8
:100190001146EA489C30FFF7B3FF14220121E748DB
:1001A0009C30FFF7ADFF14220221E4489C30FFF79A
:1001B000A7FF0C21E148C0F8A8100021C0F8AC103E
:1001C000C0F8B0101E2200F59C70FFF799FF1E22A8
:1001D0000121DB48FFF794FF1E220221D848FFF7D8
:1001E0008FFF1221D548C0F844110021C0F84811F2
:1001F000C0F84C1110BD00B589B0D24840690090DC
:10020000D0480369D0A1C26801A803F0A9F910235E
:1002100001AA0021084601F0ACF809B000BD002198
:10022000CC4A1160CC4AC2F8B411CC4A1160CC4A15
:10023000C2F8AC11C0EBC00101EB4011BF4A02EBA8
:100240008101096D002902DD0121C24A1160C0EB64
:10025000C00101EB4011B94A02EB8101496F00294D
:1002600003DD0121BB4A121F1160C0EBC00101EB8D
:100270004011B24A02EB8101D1F89810002902DD49
:100280000121B64A1160704710B50020B149091D1F
:100290000860642001F0CFFA0120AF49C1F8BC0129
:1002A00010BD0021012200BF36E0C1EBC10000EB10
:1002B0004110A24B03EB8000C068A24BDB68984260
:1002C00001D0002220E0C1EBC10000EB41109B4BAC
:1002D00003EB800000699B4B1B69984204D000220D
:1002E0000020A04B18600FE0C1EBC10000EB4110F3
:1002F000924B03EB80004069924B5B69984203D0BC
:100300009848006800B9002222B10120954B18607E
:10031000084670470122491C0329C6DB4FF0FF3015
:10032000F7E710B588B0FFF7BCFF0446601CC8B300
:10033000FFF7AAFF2046FFF772FFC4EBC40000EBF3
:1003400044107E4A02EB800000F13001684603F061
:10035000A8F8C4EBC40000EB4410784A02EB80001C
:1003600000F15401684603F07EF8C4EBC40000EBD2
:100370004410724A02EB800000F17801684603F0F5
:1003800072F810236A460221002000F0F2FF76483E
:10039000006800281AD1684601F0C7F901207249A7
:1003A000086013E0FFE7102370A20221002000F094
:1003B000E0FF0020674908606749C1F8B401674958
:1003C000086066490C3108606749086008B010BDD4
:1003D00010B501F0F3F94FF4A06002F0A5F84FF466
:1003E000E13001F079FA00F061FA01F051F801F022
:1003F0007EF96B4800F09DFD00F0E1FEFFF7B1FED5
:1004000010BDFFF7E5FF4FF47A7001F014FA0120F8
:100410005049091D086008E000F0AEFDFFF781FFBC
:10042000FFF7E9FEC82001F006FAF5E72DE9F041F3
:1004300000270026002400255AA15B4803F01FF87E
:100440005949471A59A1584803F019F85649461A0C
:1004500000BF7C1C07E05448005D303805EB850187
:1004600000EB4105641CB442F5DB2846BDE8F08191
:10047000024600214E480088C0F30D0300BF06E08D
:100480004948405C904201D108467047491C994256
:10049000F6DB0020F9E710B5024600200021444CAD
:1004A0002488C4F30D0300BF05E03F4C645C944214
:1004B00000D10846491C9942F7DB10BD2DE9F041F7
:1004C0008CB08046002600270024002535A1364840
:1004D00002F0D5FF3449461A2D20FFF7C9FF074621
:1004E000741C07E03048005D303805EB850100EBF7
:1004F0004105641CBC42F5DB009500252D20FFF76B
:10050000B7FF06462D20FFF7C6FF0746741C59E0CB
:10051000312E416D696B696E3A2564200000000040
:10052000322E52756C69643A25642000332E427273
:100530007566656E3A256420000000008801002081
:10054000C00200205C0300202532643A2532643A60
:1005500025326400B801224200002242A00121425B
:10056000000021420C000020080000202020202054
:10057000202020202020202020202020202020207B
:10058000202020202020202020202020202020206B
:10059000202020202020202020202020202020007B
:1005A0000000002028000000F003002029000000C7
:1005B000700100203C48005D303805EB850100EB00
:1005C0004105641CBC42F5DB019500252D20FFF799
:1005D00062FF06462020FFF74BFF0746741C07E02A
:1005E0003148005D303805EB850100EB4105641CA6
:1005F000BC42F5DB029500252020FFF739FF0646B7
:100600003A20FFF735FF0746741C07E02648005DD7
:10061000303805EB850100EB4105641CBC42F5DB7D
:10062000039500253A20FFF723FF06463A20FFF7FF
:1006300032FF0746741C07E01B48005D303805EBAD
:10064000850100EB4105641CBC42F5DB04950025E7
:100650003A20FFF720FF06462920FFF71CFF074638
:10066000741C07E01048005D303805EB850100EB95
:100670004105641CBC42F5DB0595302269464046C5
:1006800002F0CDFE0CB0BDE8F08110B5074800883F
:1006900000F4004030B1C821034802F0D9FE002028
:1006A0000249088010BD0000F00300207001002006
:1006B000704700BFFEE700BFFEE700BFFEE700BFD8
:1006C000FEE7704770477047704700000CB5002088
:1006D000019000906C48006840F480306A490860DE
:1006E00000BF6948006800F4003000900198401C89
:1006F0000190009818B90198B0F5A06FF1D1624847
:10070000006800F4003010B10120009001E00020EA
:1007100000900098012843D15C48006840F0100028
:100720005A4908600846006820F00300086008463F
:10073000006840F002000860534840685249486031
:100740000846406848600846406840F48060486059
:100750000846406820F47C1048600846406840F431
:10076000E81048600846006840F08070086000BFEC
:100770004548006800F000700028F9D04248406801
:1007800020F00300404948600846406840F00200FD
:10079000486000BF3C48406800F00C000828F9D1D0
:1007A0000CBD10B5FFF792FF10BD10B536480068BC
:1007B00040F0010034490860084640683449084068
:1007C0003149486008460068324908402E490860AF
:1007D0000846006820F4802008600846406820F43D
:1007E000FE0048604FF41F008860FFF7DAFF4FF00B
:1007F00000602949086010BD10B5002100200022CA
:10080000214B5B6803F00C0121B1042906D00829B3
:1008100028D107E0214B224C236027E01F4B204CBE
:10082000236023E0184B5B6803F47010164B5B6881
:1008300003F48032022303EB904022B9194B434367
:10084000174C23600DE0104B5B6803F4003323B1B9
:10085000144B4343124C236003E0104B4343104CB2
:10086000236003E00D4B0E4C236000BF00BF064B1E
:100870005B68C3F303130C4CE15C094B1B68CB4072
:10088000074C236010BD0000001002400020024011
:100890000000FFF8FFFFF6FE08ED00E000127A000E
:1008A0001000002000093D001400002008B50121BF
:1008B000142001F0D1FB4FF46040ADF8000010208F
:1008C0008DF8030003208DF802006946054801F009
:1008D00007F94FF41060ADF800006946024801F0D6
:1008E000FFF808BD001001400008014010B586B0B7
:1008F00004460121082001F0AFFB0121880401F02A
:10090000B8FB4FF48060ADF8140003208DF816009A
:1009100018208DF8170005A9874801F0E1F84FF479
:100920000060ADF8140004208DF8170005A9824876
:1009300001F0D6F827208DF8000000208DF8010086
:1009400003208DF8020001208DF80300684601F0B5
:10095000F0FD01940020ADF80800ADF80A00ADF8F4
:100960000C00ADF810000C20ADF80E0001A9734882
:1009700001F019FC012240F22551704801F0ABFC56
:1009800001216E4801F09BFC06B010BD10B500249B
:100990006A4801F005FDC4B269486A4909784454BF
:1009A00068480078401C6749087008460078642849
:1009B00001DB0020087010BD002004E00021604A27
:1009C0001154411C88B26428F8DB00215D4A117083
:1009D000704710B504460BE000BF4021574801F0B6
:1009E00049FD0028F9D014F8011B544801F0D4FC4B
:1009F00020780028F0D110BD10B50446FFF7DCFFC9
:100A00002046FFF7E6FF50A0FFF7E3FF10BD10B54B
:100A1000044621464A4802F032FD08B1012010BDCB
:100A20000020FCE72DE9F04180460C4615461E46A5
:100A300000270EE04046FFF7DFFFB0B200F0FBFEFC
:100A40002046FFF7E4FF10B10120BDE8F081781CDB
:100A5000C7B2AF42EEDB0020F7E710B564230322F4
:100A60003AA13BA0FFF7DEFF04464FF4167000F0FA
:100A7000E2FE14B94FF0FF3010BD6423032233A10E
:100A800035A0FFF7CFFF04464FF4167000F0D3FEF9
:100A900014B96FF00100EFE7642303222BA132A009
:100AA000FFF7C0FF04464FF4167000F0C4FE14B9FF
:100AB0006FF00200E0E76423032224A132A0FFF7D5
:100AC000B1FF04464FF4167000F0B5FE14B96FF094
:100AD0000300D1E7642303221CA12FA0FFF7A2FF8C
:100AE00004464FF4167000F0A6FE14B96FF004002F
:100AF000C2E76423032215A12DA0FFF793FF04464C
:100B00004FF4167000F097FE14B96FF00500B3E7CC
:100B10000020B1E710B504463223032228A129A002
:100B2000FFF780FFC82000F086FE2046FFF751FF48
:100B3000642000F080FE10BD000C01400048004021
:100B40008C030020240000200D0000004F4B00000B
:100B500041540D0A0000000041542B43574D4F44AF
:100B6000453D320D0A00000041542B43575341507C
:100B70003D225A48222C2231323334353637383927
:100B8000222C352C330D0A0041542B4349504D552E
:100B9000583D310D0A00000041542B434950534544
:100BA000525645523D312C353030300D0A00000090
:100BB00041542B43495053544F3D300D0A0000001F
:100BC0003E00000041542B43495053454E443D30B4
:100BD0002C31340D0A0000007FB505460C4601217A
:100BE000022001F046FAADF80850ADF804400020AC
:100BF000ADF80A00ADF8060001A9334801F0D6FDB2
:100C000001221146304802F048F91D208DF80000FD
:100C100003208DF801008DF8020001208DF80300FB
:100C2000684601F086FC0121274802F01BF97FBDD0
:100C300010B50121244802F0DEFB18B10121224841
:100C400002F0EAFB10BD30B589B005460C46012123
:100C5000022001F00EFA0121092001F0FDF9012125
:100C60001A4801F00EF80220ADF8200018208DF887
:100C7000230003208DF8220008A9154800F030FF5A
:100C8000ADF81850ADF814400020ADF81A00ADF8DA
:100C9000160005A90C4801F089FD7020ADF804008C
:100CA0000120ADF806000020ADF80C0001A90648AF
:100CB00001F0FBFD0821044802F00DFA0121024871
:100CC00002F0D0F809B030BD0004004000081A005E
:100CD000000C014008B50121082001F0BDF9E02019
:100CE000ADF8000003208DF8020010208DF80300FD
:100CF0006946B14800F0F4FE08BD38B50446012C41
:100D00000DD14020ADF8000003208DF80200102026
:100D10008DF803006946A84800F0E2FE0DE064B9D2
:100D20004020ADF8000003208DF8020048208DF827
:100D300003006946A04800F0D3FE38BD07E06E21ED
:100D400001E04A1ED1B20029FBDC421ED0B20028CD
:100D5000F5DC7047F0B504460D4626462F46802048
:100D6000954910310860002319E006F0010020B118
:100D7000402091491031086003E040208E49143131
:100D80000860761020208C49103108600220FFF79F
:100D9000D5FF2020884914310860581CC3B2082BA5
:100DA000E3DB002319E007F0010020B14020824975
:100DB0001031086003E040207F49143108607F1043
:100DC00020207D49103108600220FFF7B7FF202066
:100DD000794914310860581CC3B2082BE3DB80202A
:100DE000754914310860F0BD2DE9F04706463746D5
:100DF0008020714910310860002519E007F00100DA
:100E000020B140206C491031086003E040206A495D
:100E1000143108607F1020206749103108600220DB
:100E2000FFF78CFF2020644914310860681CC5B2AC
:100E3000082DE3DB0020FFF760FF002517E06410BA
:100E400040215D4800F0DFFE10B144F0800401E075
:100E500004F07F0420205849103108600220FFF779
:100E60006DFF2020544914310860681CC5B2082D5C
:100E7000E5DB80205049143108600120FFF73DFF79
:100E80002046E11704EB1171C1F30718E11704EBD9
:100E900011710911A4EB011101F0FF0908EB8800A1
:100EA00009EB400000F0FF0A5046BDE8F08710B59E
:100EB000044600218E20FFF74DFF61798020FFF767
:100EC00049FF21798220FFF745FFE1788420FFF771
:100ED00041FFA1788620FFF73DFF61788820FFF76A
:100EE00039FF21788C20FFF735FF80218E20FFF716
:100EF00031FF10BD10B58120FFF776FF04460021B9
:100F00008E20FFF727FF44F0800421468020FFF762
:100F100021FF10BD10B58120FFF766FF04460021B8
:100F20008E20FFF717FF00BF21468020FFF712FF3A
:100F300010BD10B50446FFF7CDFE0220FFF7FEFE00
:100F400080201D49143108602020086000218E2077
:100F5000FFF700FFA7219020FFF7FCFE80218E20E5
:100F6000FFF7F8FE8120FFF73FFF00F0800010B18F
:100F70002046FFF79CFF10BD10B58D20FFF734FF12
:100F80000E4908608920FFF72FFF0C494860872031
:100F9000FFF72AFF094988608520FFF725FF0749E9
:100FA000C8608320FFF720FF044908618120FFF714
:100FB0001BFF0249486110BD000C01405C0300208A
:100FC00010B54FF40051F94800F037FE4FF40041DE
:100FD000F64800F032FE4FF40041F44800F02FFED6
:100FE0004FF40051F14800F02AFE10BD10B54FF447
:100FF0000051EE4800F021FE4FF40041EB4800F0B4
:101000001EFE4FF40041E94800F017FE10BD10B578
:101010004FF40051E54800F010FE4FF40051E34852
:1010200000F00DFE10BD2DE9F04105462C464FF4B1
:101030000051DE4800F003FE00261CE0274607F0C2
:101040008007802F04D13902D84800F0F6FD04E073
:101050004FF40041D54800F0F2FD6006040E4FF455
:101060000051D24800F0E9FD4FF40051CF4800F0A4
:10107000E6FD701CC6B2082EE0DBBDE8F08110B5BD
:101080000446FFF79DFF7820FFF7CDFFFFF7BFFF76
:101090000020FFF7C8FFFFF7BAFF2046FFF7C3FFA6
:1010A000FFF7B5FFFFF7A2FF10BD10B50446FFF72D
:1010B00087FF7820FFF7B7FFFFF7A9FF4020FFF772
:1010C000B2FFFFF7A4FF2046FFF7ADFFFFF79FFF3A
:1010D000FFF78CFF10BD70B504460D461DB1E0B2A0
:1010E000FFF7E3FF02E0E0B2FFF7C9FF70BD70B5A4
:1010F0000646002418E004F1B0000021FFF7EBFFE2
:1011000000210846FFF7E7FF00211020FFF7E3FF6B
:10111000002505E001213046FFF7DDFF681CC5B260
:10112000802DF7DB601CC4B2082CE4DB70BD06E048
:1011300041F6650100E0491E0029FCD1401E00284F
:10114000F6D17047014605E0002001E0421CD0B214
:101150007B28FBDB0A1EA1F10101F5D1704770B5B8
:1011600004460D4605F1B0000021FFF7B4FF102141
:1011700041EA14100021FFF7AEFF04F00F00002138
:10118000FFF7A9FF70BD10B500218D20FFF7A3FF69
:1011900000211420FFF79FFF0021AF20FFF79BFFE6
:1011A00010BD10B500218D20FFF795FF0021102004
:1011B000FFF791FF0021AE20FFF78DFF10BD70B546
:1011C000002418E004F1B0000021FFF784FF0021A3
:1011D0000846FFF780FF00211020FFF77CFF002565
:1011E00005E001210020FFF776FF681CC5B2802DC5
:1011F000F7DB601CC4B2082CE4DB70BD70B50024C2
:1012000018E004F1B0000021FFF765FF0021084657
:10121000FFF761FF00211020FFF75DFF002505E0CB
:1012200001210846FFF757FF681CC5B2802DF7DB88
:10123000601CC4B2082CE4DB70BD2DE9F047074602
:101240000E469046994600250024A8F12000C5B21C
:101250007F2F02DD0027B01CC6B2B9F1100F24D1D8
:1012600031463846FFF77BFF002408E004EB051108
:101270004F4A505C0121FFF72EFF601CC4B2082CBE
:10128000F4DB701CC1B23846FFF769FF002409E0A7
:1012900004EB05110831464A505C0121FFF71BFFA2
:1012A000601CC4B2082CF3DB12E031463846FFF76D
:1012B00056FF00240AE005EB45013E4A02EB4101DE
:1012C000085D0121FFF707FF601CC4B2062CF2DBAA
:1012D000BDE8F08710B50246012000E050430B1E28
:1012E000A1F10104E1B2F9D110BD2DE9FF5F07467C
:1012F00091461E460E9D4FF0000A002435E0301B3B
:10130000401EC1B20A20FFF7E5FFB9FBF0F00A2149
:10131000B0FBF1F201FB1208BAF1000F14D1701EFC
:10132000A04211DDB8F1000F0CD1AB4605EBDB712B
:10133000491001FB0471C8B22B4620220199FFF726
:101340007CFF10E04FF0010AAB4605EBDB71491062
:1013500001FB0471C8B208F13001CAB22B460199F1
:10136000FFF76BFF00BF601CC4B2B442C7DBBDE82F
:10137000FF9F2DE9F04104460F461546984600268A
:101380000FE0AA5D434639462046FFF756FF04F1B9
:101390000800C4B2782C02DD0024B81CC7B2701C4F
:1013A000C6B2A85D0028ECD1BDE8F081000C014078
:1013B0001C3B0008F43800082DE9F04180460E4639
:1013C0001546002731464046FFF7C9FE00240AE0D3
:1013D000744A02EB8511085D0121FFF77CFE781C41
:1013E000C7B2601CC4B2102CF2DB701CC1B2404604
:1013F000FFF7B5FE00240CE06900491C694A02EBC6
:101400004111085D0121FFF766FE781CC7B2601C20
:10141000C4B2102CF0DBBDE8F0812DE9F05F064688
:101420000F4690461C46DDF828A04FF0000BE11750
:1014300004EB5171C910A4EBC10131B92046E11789
:1014400004EB5171C1F3C70506E02046E11704EB38
:101450005171C910491CCDB23D4615E029463046B0
:10146000FFF77DFEB1460BE059460BF1010B1AF870
:1014700001000121FFF72FFE09F1010000F0FF0933
:10148000C145F1DB681CC5B2A542E7DBBDE8F09FB2
:1014900008B50121082000F0DFFD4FF42040ADF831
:1014A000000010208DF8030003208DF8020069462B
:1014B0003D4800F015FB4FF420413B4800F0BDFBD8
:1014C0004FF4487000F0B7F90021AE20FFF703FE9B
:1014D00000210846FFF7FFFD00211020FFF7FBFD6C
:1014E00000214020FFF7F7FD0021B020FFF7F3FDBA
:1014F00000218120FFF7EFFD0021FF20FFF7EBFD2A
:101500000021A120FFF7E7FD0021A620FFF7E3FD62
:101510000021A820FFF7DFFD00213F20FFF7DBFDC2
:101520000021C820FFF7D7FD0021D320FFF7D3FD0E
:1015300000210846FFF7CFFD0021D520FFF7CBFDA6
:1015400000218020FFF7C7FD0021D820FFF7C3FD51
:1015500000210520FFF7BFFD0021D920FFF7BBFDCB
:101560000021F120FFF7B7FD0021DA20FFF7B3FDDE
:1015700000211220FFF7AFFD0021DB20FFF7ABFDBC
:1015800000213020FFF7A7FD00218D20FFF7A3FDEC
:1015900000211420FFF79FFD0021AF20FFF79BFDE6
:1015A00008BD000025000020000C014000220021A1
:1015B00007E0002200E0521C4FF6FF739A42FAD374
:1015C000491C8142F5D3704770B50646304601F09C
:1015D000B7FF0220FFF7EAFF5F48008800F40040F1
:1015E000C8B15D480088C0F30D0500240CE05B48DD
:1015F000005D4F2806D15949601C085C4B2801D179
:10160000002070BD601C84B2AC42F0DB0020524967
:1016100008800120F5E70120F3E770B50646304663
:1016200001F08EFF0220FFF7C1FF4B48008800F455
:101630000040F8B148480088C0F30D0500240EE0D2
:101640004648005D3E2808D1002043490880C82153
:10165000424801F0FDFE002070BD601C84B2AC4227
:10166000EEDB00203C490880C8213C4801F0F0FE38
:101670000120F1E70120EFE770B50646304601F0A2
:101680005FFF0220FFF792FF1A21354800F084FE29
:101690000220FFF78BFF3048008800F4004020B3A1
:1016A0002D480088C0F30D05002413E02B48005D91
:1016B0004F280DD12949601C085C4B2808D1002017
:1016C00025490880C821254801F0C2FE002070BDD0
:1016D000601C84B2AC42E9DB00201F490880C821AD
:1016E0001E4801F0B5FE0120F1E70120EFE710B53B
:1016F0001CA0FFF769FF0020174908801CA0FFF716
:1017000063FF0020144908801DA0FFF75DFF002043
:101710001149088020A0FFF757FF00200E490880DC
:101720004FF47A7000F087F810BD10B504461DA084
:10173000FFF74AFF0020084908800220FFF736FF24
:101740002046FFF741FF1A21054800F025FE002042
:101750000149088010BD000070010020F003002046
:101760000038014041542B434D47463D310D0A009E
:1017700041542B435343533D2247534D220D0A00FE
:1017800041542B43534D503D31372C3136372C309B
:101790002C3234300D0A000041542B434D47443D58
:1017A000310D0A0041542B434D47533D2231313115
:1017B0003131313131313131220D0A0010B56FF044
:1017C000040000F000FF2E4800682E49B0FBF1F045
:1017D0002D4908700846007800EB4001C1EBC010AD
:1017E0004FF6FF7101EAC0002849088010BD01468C
:1017F000254A12784A434FF0E0235A6100229A6149
:101800001A46126942F001021A6100BF4FF0E0224D
:10181000106900F001021AB100F48032002AF5D0FC
:101820004FF0E022126922F001024FF0E0231A612A
:1018300000229A6170470146144A12884A434FF0C9
:10184000E0235A6100229A611A46126942F00102AD
:101850001A6100BF4FF0E022106900F001021AB1D6
:1018600000F48032002AF5D04FF0E022126922F015
:1018700001024FF0E0231A6100229A6170470000D4
:101880001000002000127A0066010020680100208C
:10189000014600BF704700BF544A128802F0400260
:1018A000002AF9D0C2B2514B1B1D1A80704770B587
:1018B00005460E46002400BF0BE000BF40214B4808
:1018C00000F0D8FD0028F9D0295D484800F064FDFB
:1018D000641CB442F1DB70BD10B586B00446012132
:1018E00044F2040000F0B8FB4FF40070ADF81400AF
:1018F00003208DF8160018208DF8170005A93C4824
:1019000000F0EEF84FF48060ADF8140004208DF87C
:10191000170005A9364800F0E3F825208DF80000EF
:1019200003208DF801008DF8020001208DF80300DE
:10193000684600F0FEFD01940020ADF80800ADF807
:101940000A00ADF80C00ADF810000C20ADF80E0048
:1019500001A9264800F027FC012240F22551234826
:1019600000F0B9FC0121214800F0A9FC06B010BD2F
:1019700010B540F225511D4800F092FD10B31B48F0
:1019800000F00EFDC4B21B48008800F40040C8B946
:101990001848008800F4804060B10A2C03D0002071
:1019A0001449088020E01348008840F400401149A1
:1019B000088019E00D2C06D10E48008840F48040C4
:1019C0000C49088010E00B480088C0F30D000A495C
:1019D0000C5408480088401C0649088008460088C6
:1019E000C72801DD0020088010BD0000003801403C
:1019F0000008014070010020F003002006488047E5
:101A000006480047FEE7FEE7FEE7FEE7FEE7FEE7E3
:101A1000FEE7FEE7FEE7FEE7AB070008ED00000883
:101A200010B50446CC48844208D10121042000F0BE
:101A30002DFB0021042000F029FB46E0C74884422A
:101A400008D10121082000F021FB0021082000F02E
:101A50001DFB3AE0C248844208D10121102000F069
:101A600015FB0021102000F011FB2EE0BD48844240
:101A700008D10121202000F009FB0021202000F0E6
:101A800005FB22E0B848844208D10121402000F043
:101A9000FDFA0021402000F0F9FA16E0B348844234
:101AA00008D10121802000F0F1FA0021802000F00F
:101AB000EDFA0AE0AE48844207D10121801500F01A
:101AC000E5FA0021A01500F0E1FA10BD10B50121E2
:101AD000084600F0DBFA0021012000F0D7FA10BD23
:101AE0002DE9F041024600250026002000230024B5
:101AF000002791F803C00CF00F0591F803C00CF01B
:101B0000100CBCF1000F03D091F802C04CEA05059F
:101B100091F800C0BCF1000F31D0146800202BE018
:101B20004FF0010C0CFA00F3B1F800C00CEA030608
:101B30009E4220D183004FF00F0C0CFA03F7BC43F8
:101B400005FA03FC4CEA040491F803C0BCF1280F29
:101B500006D14FF0010C0CFA00FCC2F814C00AE0E8
:101B600091F803C0BCF1480F05D14FF0010C0CFAFD
:101B700000FCC2F810C0401C0828D1D31460B1F892
:101B800000C0BCF1FF0F34DD546800202EE000F1EE
:101B9000080C4FF0010808FA0CF3B1F800C00CEA89
:101BA00003069E4221D183004FF00F0C0CFA03F77D
:101BB000BC4305FA03FC4CEA040491F803C0BCF1F1
:101BC000280F05D100F1080C08FA0CF8C2F81480AF
:101BD00091F803C0BCF1480F07D100F1080C4FF099
:101BE000010808FA0CF8C2F81080401C0828CED36F
:101BF0005460BDE8F0814FF6FF71018002218170D1
:101C00000421C17070470246002093680B400BB15D
:101C1000012000E0002070470146886880B27047CC
:101C200002460020D3680B400BB1012000E00020E9
:101C300070470146C86880B27047016170474161D2
:101C400070470AB1016100E041617047C1607047AF
:101C50004FF480320A4382618161826182698269C4
:101C6000704702460020434B18684FF680731840B7
:101C700040EA021008433F4B186070473E49C86174
:101C80007047F0B50A46002300240021002500F02B
:101C90000046B6F1004F02D1364EF16901E0354EF3
:101CA0007168C0F3034583B200F44016B6F5401FD7
:101CB00008D121F070612F4E766826F070662D4FA6
:101CC0007E6012E000F48016B6F5801F06D1032670
:101CD00006FA05F4A14341F0706106E0460D3601B5
:101CE00003FA06F6B14341F0706122B1460D3601A8
:101CF00003FA06F6314300F00046B6F1004F02D178
:101D00001C4EF16101E01B4E7160F0BD30B5002248
:101D10008B071C0F0F2303FA04F2164B08338C10A9
:101D200053F824309343134C08348D1044F8253075
:101D300023468C1053F824308C07240F00FA04F447
:101D400023430C4C08348D1044F8253030BD0A492B
:101D5000DC3108607047000000080140000C0140C1
:101D6000001001400014014000180140001C014017
:101D7000002001400000014000002042DF480068D0
:101D800040F00100DD49086008464068DC49084031
:101D9000DA49486008460068DA490840D7490860CF
:101DA0000846006820F4802008600846406820F457
:101DB000FE0048604FF41F0088607047CF490968F3
:101DC00021F48031CD4A11601146096821F4802147
:101DD0001160B0F5803F03D0B0F5802F0ED106E042
:101DE000C649096841F48031C44A116007E0C3491B
:101DF000096841F4A021C14A116000E000BF00BFA2
:101E0000704710B501460022002300204A11012A24
:101E100002D1BA4C236806E0022A02D1B74C236AE9
:101E200001E0B64C636A01F01F02012494401C409B
:101E30000CB1012000E0002010BD38B5002000905A
:101E40000024002500BF3120FFF7DBFF0546009886
:101E5000401C00900098B0F5A06F01D0002DF2D08A
:101E60003120FFF7CEFF08B1012400E00024204616
:101E700038BD01460020A14A106820F0F80040EA71
:101E8000C10010607047A0490860704702460020FA
:101E90009A4B586820F47C1042EA01031843974B90
:101EA0005860704798490866704701460020934A79
:101EB000506820F003000843506070478F48406826
:101EC00000F00C007047014600208C4A506820F05A
:101ED000F00008435060704701460020874A506870
:101EE00020F4E06008435060704701460020834AB8
:101EF000506820F4605040EAC1005060704729B13A
:101F00007E4A527A02437D4B5A7204E07B4A527AEF
:101F100082437A4B5A7270477B49D83108607047C8
:101F200001460020754A506820F440400843506044
:101F300070470021714A20321170704A82F82010D7
:101F4000012802D004280AD104E001216B4A203282
:101F5000117005E00521694A2032117000E000BFD0
:101F600000BF70476949086070476449096A0143C6
:101F7000624A11627047654944390860704730B55C
:101F800000210022002400235C4D6D6805F00C0147
:101F900021B1042905D0082923D105E05C4D056055
:101FA00022E05B4D05601FE0544D6D6805F4701232
:101FB000524D6D6805F48034022505EB92421CB940
:101FC000544D554305600BE04C4D6D6805F40035EC
:101FD0001DB1504D5543056002E04D4D5543056020
:101FE00002E04B4D056000BF00BF444D6D6805F039
:101FF000F0010909484D6B5C0568DD4045603F4DC7
:102000006D6805F4E061090A434D6B5C4568DD408D
:1020100085603A4D6D6805F46051C90A3E4D6B5CB0
:102020004568DD40C560354D6D6805F44041890B5C
:102030003A4D6B5CC568B5FBF3F5056130BD29B160
:102040002E4A526902432D4B5A6104E02B4A5269D1
:1020500082432A4B5A61704729B1284A9269024348
:10206000264B9A6104E0254A92698243234B9A6188
:10207000704729B1214AD2690243204BDA6104E05A
:102080001E4AD26982431D4BDA61704729B11B4A4F
:10209000D2680243194BDA6004E0184AD2688243DE
:1020A000164BDA60704729B1144A12690243134B88
:1020B0001A6104E0114A12698243104B1A61704799
:1020C00012494039086070470F49C86470470B498E
:1020D000C87170470948406A40F0807007494862FB
:1020E000704701460020054A92680A400AB1012063
:1020F00000E00020704701498872704700100240DC
:102100000000FFF8FFFFF6FE00004242800442425A
:1021100000127A0000093D007201002082010020B7
:1021200010B50446FB48844209D101218803FFF71A
:10213000ADFF00214FF48040FFF7A8FF32E0F648E2
:10214000844209D101214804FFF7ADFF00214FF47B
:102150000030FFF7A8FF25E0F048844209D10121B3
:102160008804FFF7A0FF00214FF48020FFF79BFFBA
:1021700018E0EB48844209D10121C804FFF793FF1E
:1021800000214FF40020FFF78EFF0BE0E54884426A
:1021900008D101210805FFF786FF00214FF48010C8
:1021A000FFF781FF10BD2DE9F04786B005460E46CA
:1021B0000024A24600BFA1460027B08900B100BF9D
:1021C0002F462C8A4CF6FF700440F08804432C8282
:1021D000AC894EF6F3100440B08831890843718908
:1021E00008430443AC81AC8A4FF6FF400440B089F9
:1021F0000443AC8201A8FFF7C2FEC648874202D161
:10220000DDF810A001E0DDF80CA0A88900F4004082
:1022100040B10AEBCA0000EB0A1031684900B0FB7C
:10222000F1F807E00AEBCA0000EB0A1031688900F8
:10223000B0FBF1F86420B8FBF0F004012009642140
:1022400001FB1089A88900F4004040B1322000EB66
:10225000C900B0FBF1F000F00700044308E03220B1
:1022600000EB09106421B0FBF1F000F00F00044313
:102270002C8106B0BDE8F0874FF4165101600021B3
:102280008180C18001810C214181002181817047C1
:1022900010B502460020108A4FF2FF0318400B8849
:1022A0004C8823438C882343CC88234318431082D3
:1022B00010BD0021018041808180C180704721B123
:1022C000828942F40052828104E082894DF6FF73D4
:1022D0001A4082817047F0B503460024002600258D
:1022E000002040F66A17B94200D100BF1846C1F37A
:1022F000421401F01F06012707FA06F5012C01D14F
:102300000C3004E0022C01D1103000E014301AB17E
:1023100007682F43076002E00768AF430760F0BD1E
:102320001AB1838A0B43838202E0838A8B438382C0
:102330007047028A4FF6F0731A400282028A0A43FB
:102340000282704782894FF2FF731A40828182892C
:102350000A438281704721B1828942F00202828160
:1023600004E082894FF6FD731A4082817047028A29
:102370004FF6DF731A400282028A0A4302827047D4
:1023800021B1028A42F48042028204E0028A4BF6C2
:10239000FF731A4002827047C1F3080282807047BF
:1023A00001468888C0F308007047818941F0010127
:1023B00081817047028BD2B20283028B42EA0122F2
:1023C00002837047028B02F47F420283028B0A432E
:1023D0000283704721B1828A42F02002828204E0A7
:1023E000828A4FF6DF731A408282704721B1828A57
:1023F00042F01002828204E0828A4FF6EF731A40A4
:102400008282704721B1828A42F00802828204E00F
:10241000828A4FF6F7731A408282704721B182890F
:1024200042F40042828103E08289C2F30E0282817B
:10243000704721B1828A42F40062828204E0828A7B
:102440004FF2FF731A4082827047828A4FF6FB7305
:102450001A408282828A0A438282704721B1828A2C
:1024600042F00202828204E0828A4FF6FD731A4033
:102470008282704702460020B1F5007F00D100BF84
:1024800013880B400BB1012000E00020704701F4DD
:102490000072B2F5007F00D100BFCA4302807047CE
:1024A00070B50246002400230025002040F66A167D
:1024B000B14200D100BFC1F3421501F01F03012654
:1024C00006FA03F3012D02D19689334006E0022D6E
:1024D00002D1168A334001E0968A33400C1201265D
:1024E00006FA04F41688344013B10CB1012000E060
:1024F000002070BD10B50022002340F66A14A142EE
:1025000000D100BF0A1201249440A3B2DC4304802E
:1025100010BD000000380140004400400048004069
:10252000004C00400050004031490143314A1160E5
:10253000704770B5002100230F22C47804B32D4CDE
:10254000246804F4E064C4F5E064210AC1F10403E2
:10255000CA40447804FA03F1847814402143090105
:10256000254C0678A155047804F01F050124AC40E1
:1025700005786D11AD0005F1E025C5F8004109E0D1
:10258000047804F01F050124AC401C4D0678761138
:1025900045F8264070BD1A4A0A400243154B1B1FDE
:1025A0001A60704739B1134A121D12680243114B69
:1025B0001B1D1A6006E00F4A121D126882430D4B64
:1025C0001B1D1A607047042808D14FF0E0210969EB
:1025D00041F004014FF0E022116107E04FF0E021EB
:1025E000096921F004014FF0E022116170470000F9
:1025F0000000FA050CED00E000E400E080E100E0FE
:1026000080FFFF1F10B50446FE48844208D1012117
:10261000C014FFF73BFD0021E014FFF737FDC4E0D5
:10262000B4F1804F08D101210846FFF73CFD00219D
:102630000120FFF738FDB8E0F348844208D10121BA
:102640000220FFF730FD00210220FFF72CFDACE057
:10265000EE48844208D101210420FFF724FD002127
:102660000420FFF720FDA0E0E948844208D10121C1
:102670000820FFF718FD00210820FFF714FD94E063
:10268000E448844208D101211020FFF70CFD00210D
:102690001020FFF708FD88E0DF48844208D10121BF
:1026A0002020FFF700FD00212020FFF7FCFC7CE04C
:1026B000DA48844208D101214014FFF7E7FC0021E9
:1026C0006014FFF7E3FC70E0D548844209D1012192
:1026D000C804FFF7DBFC00214FF40020FFF7D6FC15
:1026E00063E0D048844209D101210805FFF7CEFC00
:1026F00000214FF48010FFF7C9FC56E0CA4884421D
:1027000009D101214805FFF7C1FC00214FF4001059
:10271000FFF7BCFC49E0C548844208D101214020B4
:10272000FFF7C1FC00214020FFF7BDFC3DE0C048A1
:10273000844208D101218020FFF7B5FC00218020D0
:10274000FFF7B1FC31E0BB48844208D1012180157C
:10275000FFF7A9FC0021A015FFF7A5FC25E0B6486E
:10276000844209D101210804FFF790FC00214FF4B5
:102770008030FFF78BFC18E0B048844209D101217A
:102780004804FFF783FC00214FF40030FFF77EFC84
:102790000BE0AB48844208D101218804FFF776FCA6
:1027A00000214FF48020FFF771FC10BD0022028849
:1027B000944B98420ED0994B98420BD0B0F1804F79
:1027C00008D0914B984205D0904B984202D0904B44
:1027D000984204D14FF68F731A404B881A438D4BA1
:1027E000984207D08C4B984204D04FF6FF431A40D2
:1027F000CB881A4302808B8883850B880385814BA5
:1028000098420BD0854B984208D08B4B984205D00C
:102810008A4B984202D08A4B984201D10B7A0386A8
:1028200001238382704770B5002400220023058CA9
:102830004FF6FE7635400584028C8388048B4FF674
:102840008F752C40B51E2C400D882C43751E2A40D8
:102850000D892A434D882A436A4DA8420BD06F4DFB
:10286000A84208D0744DA84205D0744DA84202D0A9
:10287000734DA84213D14FF6F7752A404D892A436C
:102880004FF6FB752A408D882A434FF6FF652B4093
:102890004FF6FF552B408D892B43CD892B438380E9
:1028A0000483CD888586028470BD70B50024002223
:1028B0000023058C4FF6EF7635400584028C838823
:1028C000048B48F6FF752C404FF6FF452C400D88D1
:1028D0004FF6FF7606EA05252C434FF6DF752A40B2
:1028E0000D8906EA05152A434D8806EA05152A438F
:1028F000444DA84202D0494DA8421DD14FF67F75E4
:102900002A404D894FF6FF7606EA05152A434FF611
:10291000BF752A408D8806EA05152A434FF6FF3514
:102920002B404FF2FF752B408D8906EA85052B431E
:10293000CD8906EA85052B4383800483CD880587EE
:10294000028470BD70B5002400220023058C4FF670
:10295000FF6635400584028C8388848B4FF68F7523
:102960002C404FF6FC752C400D882C434FF6FF553C
:102970002A400D894FF6FF7606EA05252A434D8841
:1029800006EA05252A431F4DA84202D0234DA8423E
:102990001DD14FF2FF752A404D894FF6FF7606EAAA
:1029A00005252A434FF6FF352A408D8806EA05257E
:1029B0002A434EF6FF752B404DF6FF752B408D894F
:1029C00006EA05152B43CD8906EA05152B438380BE
:1029D0008483CD888587028470BD70B50022002372
:1029E0000024058C4EF6FF7635400584038C8488E0
:1029F000828B48F6FF752A404FF6FF452A400D8826
:102A000020E00000002C01400004004000080040CD
:102A1000000C004000100040001400400034014051
:102A2000004C01400050014000540140001800409B
:102A3000001C0040002000400040014000440140D4
:102A4000004801404FF6FF7606EA05252A434DF679
:102A5000FF752B400D8906EA05352B434D8806EAA4
:102A600005352B43FA4DA84202D0FA4DA84208D1B1
:102A70004BF6FF752C408D894FF6FF7606EA8515DB
:102A80002C4384808283CD88A0F84050038470BD9D
:102A9000828B4FF2FF331A408283828B4FF6FF7393
:102AA00003EA01231A4382837047F0B50C461546AA
:102AB000002200210026078C4EF6FF7C07EA0C0757
:102AC0000784828B018C4FF6FF7707EA043640F6C5
:102AD000FF473A404FF6FF7707EA05273A434FF69C
:102AE000FF7707EA03373A43D94FB8420ED0D94FA0
:102AF000B8420BD0B0F1804F08D0D74FB84205D0C4
:102B0000D64FB84202D0D64FB84206D14DF6FF7725
:102B1000394046F48057394305E047F6FF573940BE
:102B200044F48057394382830184F0BD828B4FF691
:102B3000F3731A408283828B0A4382837047F0B515
:102B40000C461546002200210026078C4FF6FF6C2C
:102B500007EA0C070784828B018C4FF6FF7707EAA0
:102B600004264FF60C773A404FF6FF7707EA031733
:102B70002F433A43B64FB8420ED0B64FB8420BD0AF
:102B8000B0F1804F08D0B44FB84205D0B34FB8422F
:102B900002D0B34FB84206D14FF6FF57394046F442
:102BA0008077394305E04FF2FF57394044F480778E
:102BB000394382830184F0BD028B4FF2FF331A4008
:102BC0000283028B4FF6FF7303EA01231A43028349
:102BD0007047F0B50C461546002200210026078CF0
:102BE0004FF6EF7C07EA0C070784028B018C4FF647
:102BF000FF7707EA041640F6FF473A404FF6FF77A3
:102C000007EA03373A434FF6FF7707EA05273A43C7
:102C10008F4FB8420ED08F4FB8420BD0B0F1804FDB
:102C200008D08D4FB84205D08C4FB84202D08C4F9F
:102C3000B84206D14FF6DF77394046F010073943E6
:102C400005E04FF65F77394044F0100739430283BF
:102C50000184F0BD028B4FF6F3731A400283028B9E
:102C60000A4302837047F0B50C4615460022002146
:102C7000068C4FF6FE773E400684028B018C4FF6A1
:102C80000C7632407E1C06EA03162E433243704E09
:102C9000B0420ED06F4EB0420BD0B0F1804F08D092
:102CA0006D4EB04205D06D4EB04202D06C4EB04277
:102CB00006D14FF6FD76314044F00106314305E080
:102CC0004FF6F576314044F001063143028301842A
:102CD000F0BD70B505460C465D4885420ED05D4896
:102CE00085420BD0B5F1804F08D05B48854205D0B6
:102CF0005A48854202D05A48854200D100E000BFC0
:102D0000208850B92389A28861882846FFF7ABFF45
:102D1000E1882846FFF79EFF25E0208804280AD195
:102D20002389A28861882846FFF753FFE188284657
:102D3000FFF742FF17E0208808280AD12389A288DC
:102D400061882846FFF7FBFEE1882846FFF7EEFE84
:102D500009E02389A28861882846FFF7A6FEE1885A
:102D60002846FFF795FE70BD2DE9F04105460C465B
:102D700000260127608808B9022600E00026A08806
:102D8000012801D1022700E001272088A0B923896A
:102D9000A28861882846FFF766FFE1882846FFF78A
:102DA00059FF23893A4631462846FFF712FFE1884A
:102DB0002846FFF701FF13E02389A288618828468F
:102DC000FFF707FFE1882846FFF7F6FE23893A461A
:102DD00031462846FFF747FFE1882846FFF73AFFCC
:102DE000BDE8F0810A884B881A438B881A43CB8848
:102DF0001A430B891A434B891A438B891A43A0F84B
:102E0000442070474FF6FF71818000210180C1800E
:102E10004180017270470021018041808180C18022
:102E2000018141818181C181704700210180418000
:102E3000012181800021C180018170470021018032
:102E400041808180C1800181418181817047000082
:102E5000002C014000340140000400400008004004
:102E6000000C004021B1028842F00102028004E01F
:102E700002884FF6FE731A400280704731B1B0F8F5
:102E8000442042F40042A0F8442005E0B0F8442079
:102E9000C2F30E02A0F8442070471AB183890B4395
:102EA000838102E083898B438381704781827047ED
:102EB00041EA0203A0F8483070471AB183890B43F6
:102EC000838102E083898B438381704701894FF6B8
:102ED000F8721140018170470A46002101894FF6BE
:102EE0008F73194011430181704730B504460D4678
:102EF00029462046FFF7F0FF208940F00700208197
:102F000030BD2DE9F04104460D4616461F46602DA2
:102F100006D13B46012231462046FFF75AFE05E026
:102F20003B46012231462046FFF79DFE29462046BA
:102F3000FFF7D2FF208940F007002081BDE8F08133
:102F400030B50C4600210189C9B24FF6FF7505EA7C
:102F50000325154325432943018130BD2DE9F04167
:102F600005460E4617469846002443463A463146E3
:102F70002846FFF7E5FF2C894FF6F870044044F02F
:102F800007044FF68F70044044F070042C81BDE8B4
:102F9000F081F0B504460D4616461F463B463246C4
:102FA00029462046FFF7CCFF208940F4804020814D
:102FB000F0BD0185828270470A46002101884FF6E4
:102FC0008F731940114301807047F0B50C461546C8
:102FD0001E460021002200230189028B038C4FF63C
:102FE000F877394021434FF6FC473A4040F2011749
:102FF0003A434FF6DD773B404FF6FF7707EA061777
:103000002F433B43018102830384F0BD0A46002124
:10301000018B4FF68F7319401143018370470A46A5
:103020000021018B48F6FF7319404FF6FF7303EA46
:1030300002231943018370470A460021818B4FF612
:103040008F7319401143818370470A460021818B99
:1030500048F6FF7319404FF6FF7303EA0223194342
:103060008183704721B1028842F08002028004E02F
:1030700002884FF67F731A400280704721B1828820
:1030800042F00402828004E082884FF6FB731A400B
:103090008280704721B1828842F00802828004E079
:1030A00082884FF6F7731A408280704721B1828878
:1030B00042F00102828004E082884FF6FE731A40DB
:1030C000828070470A460021018B4FF6F773194042
:1030D0001143018370470A460021018B4FF2FF73B1
:1030E00019404FF6FF7303EA022319430183704727
:1030F0000A460021818B4FF6F773194011438183F3
:1031000070470A460021818B4FF2FF7319404FF63A
:10311000FF7303EA02231943818370470A460021A3
:10312000018B4FF6FB7319401143018370470A4628
:103130000021018B4FF6FF3319404FF6FF7303EA6E
:1031400002231943018370470A460021818B4FF601
:10315000FB7319401143818370470A460021818B1C
:103160004FF6FF3319404FF6FF7303EA022319436A
:10317000818370470A460021018B4FF67F73194007
:103180001143018370470A460021018BC1F30E01F0
:103190004FF6FF7303EA02231943018370470A467F
:1031A0000021818B4FF67F73194011438183704753
:1031B0000A460021818BC1F30E014FF6FF7303EA2B
:1031C00002231943818370470A460021018C4FF680
:1031D000FD7319401143018470470A460021018C98
:1031E0004FF6F77319401143018470470A460021D6
:1031F000018C4FF6DF7319404FF6FF7303EA021399
:103200001943018470470A460021018C4FF67F73F1
:1032100019404FF6FF7303EA021319430184704704
:103220000A460021018C4FF6FF5319404FF6FF73F9
:1032300003EA02231943018470470A460021018CE6
:103240004FF2FF7319404FF6FF7303EA022319434D
:10325000018470470A460021018C4DF6FF73194026
:103260004FF6FF7303EA023319430184704730B508
:10327000002301248C40A3B2048C9C430484048C5E
:1032800002FA01F5ADB22C43048430BD30B5002301
:1032900004248C40A3B2048C9C430484048C02FA62
:1032A00001F5ADB22C43048430BD70B50346002057
:1032B00000241846183001258D40ACB21D8CA54362
:1032C0001D8409B1082909D100EB6100056825F0CA
:1032D000700505600568154305600EE00D1FC5F318
:1032E0004E052844056825F4E045056005684FF65D
:1032F000FF7606EA02263543056070BD21B10288DB
:1033000042F00202028004E002884FF6FD731A4088
:103310000280704721B1028842F00402028004E07A
:1033200002884FF6FB731A400280704721B18288F1
:1033300042F08002828004E082884FF67F731A4058
:103340008280704702884FF6F7731A400280028825
:103350000A430280704782884FF68F731A4082803A
:1033600082880A438280704702894FF6F8731A40B8
:10337000028102890A430281704702894FF67F73F6
:103380001A40028102890A43028170478184704792
:1033900081857047818670470187704781877047B4
:1033A000A0F84010704702884FF6FF431A40028091
:1033B00002880A43028070470146888E70470146A2
:1033C000088F70470146888F70470146B1F840006A
:1033D00070470146888C70470146088D7047024649
:1033E0000020138A0B400BB1012000E00020704741
:1033F000CA430282704730B50246002000230024F1
:10340000158A05EA0103958905EA010413B10CB197
:10341000012000E0002030BDCA430282704740EA2C
:1034200001039B0703D009E008C9121F08C0042A42
:10343000FAD203E011F8013B00F8013B521EF9D229
:103440007047D2B201E000F8012B491EFBD2704751
:103450000022F6E710B513460A4604461946FFF760
:10346000F0FF204610BD421E12F8013F002BFBD199
:1034700011F8013B02F8013B002BF9D1704730B540
:1034800005462A460B4612F8010B13F8014B08B10A
:10349000A042F8D01CB1002802D06D1CF1E72846EC
:1034A00030BD034611F8012B00F8012B002AF9D199
:1034B0001846704730B50B460146002020220124F3
:1034C00009E021FA02F59D4205D303FA02F5491BF2
:1034D00004FA02F52844151EA2F10102F1DC30BD08
:1034E000064C074D06E0E06840F0010394E8070051
:1034F00098471034AC42F6D3FCF7FCFD0C410008B1
:103500002C41000830B58C1810F8012B12F00F0375
:1035100001D110F8013B120906D110F8012B03E08C
:1035200010F8015B01F8015B5B1EF9D101E001F8C5
:10353000013B521EFBD1A142E6D3002030BD00006A
:103540000FB4054B10B503A9044A029800F02CF8FB
:1035500010BC5DF814FB0000971800086C010020F7
:103560000FB4084B10B504A902AA039800F01CF888
:10357000044602A9002000F0B8F9204610BC5DF80E
:1035800014FB0000EB38000802E008C8121F08C155
:10359000002AFAD170477047002001E001C1121FD4
:1035A000002AFBD1704700002DE9FF4F8BB0884601
:1035B0000546002606E025280BD0DDE90D129047D0
:1035C0006D1C761C28780028F5D10FB03046BDE878
:1035D000F08F0024A146A2460122AE4900E0044338
:1035E00015F8013F203B02FA03F00842F7D1287892
:1035F0002A2810D06FF02F022878A0F13001092975
:1036000015D809EB890102EB410144F0020400EBFB
:1036100001096D1CF0E758F8041B5FEA010903D5A6
:1036200044F40054C9F1000944F002046D1C2878E8
:103630002E2817D115F8010F44F004042A280ED0C3
:103640006FF02F022878A0F1300109290AD80AEB7F
:103650008A0102EB410100EB010A6D1CF2E758F808
:1036600004AB6D1C28786C280FD006DC4C2817D0D2
:1036700068280DD06A2814D104E0742810D07A2864
:103680000FD10DE044F400140AE044F4801401E08A
:1036900044F440146978814202D104F580146D1C11
:1036A0006D1C2878692865D006DC00288DD0632839
:1036B00027D0642806D15DE06E2808D073282AD070
:1036C000752877D0DDE90D129047761CE0E0C4F351
:1036D0000250022809D003280DD0D8F80010042881
:1036E0000DD00E6008F10408D2E0D8F80010F217EF
:1036F000C1E90062F6E7D8F800100E80F2E70E701C
:10370000F0E718F8041B8DF8001000208DF8010078
:10371000EB46012003E058F804BB4FF0FF3061078F
:103720004FF0000701D40AE07F1C57450DDA8742AD
:10373000FADB1BF807100029F6D106E07F1C874250
:10374000FCDB1BF807100029F8D1DDE90D23A9EBFC
:1037500007008146214600F0B1F83044C61904E064
:10376000DDE90D121BF8010B90477F1EF8D22146B0
:10377000484688E058F8040BC4F302514FF00A0B96
:10378000032900D100B2042900D140B2002802DA96
:1037900040422D2102E0210505D52B218DF8241072
:1037A000012104E006E0E10710D02021F6E708AF90
:1037B000089113E058F8040BC4F302514FF00A0BC0
:1037C000032900D180B2042900D1C0B20021EEE764
:1037D0005946FFF76FFE303107F8011D0028F7D179
:1037E000ADEB070000F1200B600702D524F4803414
:1037F00001E04FF0010ADA4502DDAAEB0B0000E020
:103800000020824600EB0B0108980144A9EB01005F
:103810000A90E00306D4DDE90D2321460A9800F062
:103820004DF806444FF0000908E009A911F8090015
:10383000DDE90D12904709F10109761C08998945C7
:10384000F3DBE0030CD5DDE90D2321460A9800F0F7
:1038500035F8064404E0DDE90D1230209047761C6F
:10386000BAF10001AAF1010AF5DC05E0DDE90D126B
:1038700017F8010B9047761CBBF10001ABF1010B6F
:10388000F4DC0A982146DDE90D2300F005F8064432
:103890006D1C97E6092801002DE9F041044600253A
:1038A0001E461746880404D405E039462020B04758
:1038B0006D1C641EF9D52846BDE8F0812DE9F04164
:1038C000044600251E469046C80301D5302700E077
:1038D0002027880404D505E041463846B0476D1CD2
:1038E000641EF9D52846BDE8F0810A68531C0B60B8
:1038F000107070470000000000000000002F000062
:1039000000000700070000147F147F1400242A7FA2
:103910002A12006264081323003649552250000021
:103920000503000000001C224100000041221C0091
:103930000014083E08140008083E0808000000A013
:10394000600000080808080800006060000000200F
:1039500010080402003E5149453E0000427F4000ED
:10396000004261514946002141454B310018141273
:103970007F10002745454539003C4A494930000140
:103980007109050300364949493600064949291E8F
:1039900000003636000000005636000000081422F1
:1039A00041000014141414140000412214080002F1
:1039B0000151090600324959513E007C1211127C16
:1039C000007F49494936003E41414122007F414143
:1039D000221C007F49494941007F09090901003E35
:1039E0004149497A007F0808087F0000417F410073
:1039F000002040413F01007F08142241007F4040E9
:103A00004040007F020C027F007F0408107F003ED0
:103A10004141413E007F09090906003E4151215EB6
:103A2000007F091929460046494949310001017FB3
:103A30000101003F4040403F001F2040201F003F49
:103A40004038403F006314081463000708700807FB
:103A500000615149454300007F41410000552A550E
:103A60002A55000041417F00000402010204004089
:103A700040404040000001020400002054545478AB
:103A8000007F4844443800384444442000384444CB
:103A9000487F00385454541800087E090102001869
:103AA000A4A4A47C007F080404780000447D4000A6
:103AB000004080847D00007F102844000000417F8A
:103AC0004000007C04180478007C08040478003866
:103AD0004444443800FC242424180018242418FCEE
:103AE000007C0804040800485454542000043F4457
:103AF0004020003C4040207C001C2040201C003C1A
:103B00004030403C004428102844001CA0A0A07C69
:103B1000004464544C4414141414141400000000A1
:103B2000000000000000000000000000000000F89D
:103B300000000000000000333000000000100C0600
:103B4000100C0600000000000000000040C078409B
:103B5000C0784000043F04043F040400007088FC67
:103B600008300000001820FF211E0000F008F000BF
:103B7000E018000000211C031E211E0000F0088830
:103B8000700000001E2123241927211010160E009A
:103B9000000000000000000000000000000000E045
:103BA000180402000000000718204000000204185A
:103BB000E00000000040201807000000404080F0B6
:103BC000804040000202010F01020200000000F0EC
:103BD000000000000101011F0101010000000000C0
:103BE0000000000080B07000000000000000000035
:103BF00000000000000101010101010100000000BE
:103C00000000000000303000000000000000000054
:103C100080601804006018060100000000E0100831
:103C20000810E000000F102020100F00001010F806
:103C3000000000000020203F202000000070080845
:103C400008887000003028242221300000300888C5
:103C5000884830000018202020110E000000C020ED
:103C600010F8000000070424243F240000F808880E
:103C7000880808000019212020110E0000E010889B
:103C800088180000000F112020110E0000380808CD
:103C9000C83808000000003F0000000000708808DD
:103CA00008887000001C222121221C0000E010085E
:103CB0000810E0000000312222110F00000000C0B7
:103CC000C000000000000030300000000000008054
:103CD0000000000000008060000000000000804044
:103CE000201008000001020408102000404040405D
:103CF00040404000040404040404040000081020B0
:103D000040800000002010080402010000704808F4
:103D10000808F0000000003036010000C030C8285C
:103D2000E810E0000718272423140B000000C03817
:103D3000E0000000203C23020227382008F8888891
:103D400088700000203F202020110E00C03008089D
:103D500008083800071820202010080008F8080874
:103D60000810E000203F202020100F0008F888886D
:103D7000E8081000203F20202320180008F8888839
:103D8000E8081000203F200003000000C0300808B1
:103D90000838000007182020221E020008F808003A
:103DA0000008F808203F210101213F20000808F801
:103DB000080800000020203F202000000000080824
:103DC000F8080800C08080807F00000008F888C0E4
:103DD00028180800203F20012638200008F8080095
:103DE00000000000203F20202020300008F8F800CC
:103DF000F8F80800203F003F003F200008F830C0DE
:103E00000008F808203F200007183F00E0100808CD
:103E10000810E0000F10202020100F0008F80808FC
:103E20000808F000203F210101010000E01008080F
:103E30000810E0000F18242438504F0008F8888834
:103E400088887000203F2000030C30200070880814
:103E5000080838000038202121221C00180808F822
:103E6000080818000000203F2000000008F80800A3
:103E70000008F808001F202020201F000878880074
:103E800000C83808000007380E010000F80800F8E4
:103E90000008F800033C0700073C0300081868808E
:103EA0008068180820302C03032C30200838C80004
:103EB000C83808000000203F200000001008080853
:103EC000C83808002038262120201800000000FEF5
:103ED000020202000000007F40404000000C30C0A1
:103EE00000000000000000010638C00000020202CD
:103EF000FE000000004040407F000000000004027F
:103F000002020400000000000000000000000000A9
:103F10000000000080808080808080800002020499
:103F20000000000000000000000000000000808091
:103F3000808000000019242222223F2008F80080FF
:103F400080000000003F112020110E0000000080C2
:103F500080800000000E1120202011000000008051
:103F60008088F800000E112020103F200000808083
:103F700080800000001F222222221300008080F097
:103F8000888888180020203F2020000000008080C2
:103F900080808000006B94949493600008F8008007
:103FA00080800000203F210000203F200080989862
:103FB000000000000020203F2020000000000080C2
:103FC0009898000000C08080807F000008F8000002
:103FD00080808000203F24022D302000000808F857
:103FE000000000000020203F202000008080808012
:103FF00080808000203F20003F20003F80800080A4
:1040000080800000203F210000203F2000008080B1
:1040100080800000001F202020201F008080008062
:104020008000000080FFA12020110E000000008011
:1040300080808000000E112020A0FF808080800002
:104040008080800020203F2120000100000080802F
:10405000808080000033242424241900008080E024
:10406000808000000000001F2020000080800000F1
:1040700000808000001F202020103F2080808000D2
:104080000080808000010E300806010080800080E2
:10409000008080800F300C030C300F000080800007
:1040A000808080000020312E0E3120008080800032
:1040B0000080808080818E701806010000808080E2
:1040C000808080000021302C222130000000000080
:1040D000807C020200000000003F40400000000021
:1040E000FF00000000000000FF0000000002027C52
:1040F000800000000040403F000000000006010179
:104100000202040400000000000000002C4100082E
:10411000000000208801000004350008F04100087C
:10412000880100203007000098350008C7220430BD
:1041300016163094A24A040019120102030406075D
:10414000080900101010FF109008888888FF8888E0
:1041500088080010130444827F01808040432C10A3
:10416000284681800E1310101010D030FF30D0126E
:104170001C101036100804020132FF06140102045C
:1041800008100D13FE222222FE00FE828292A29EC1
:104190002880601F0242827F0814FF402F102C43AA
:1041A000800B1590884C57A42454548C8400101311
:1041B00001018042221A07024282423E0101010EA1
:1041C0001504E4242CB4252624B42C24E4040C2562
:1041D000FF02011E1212121E41827F3011010203E2
:1041E000040102030406070809020406080000008F
:04000005080000ED02
:00000001FF
